:10000000020C23AAAAAAAAAAAAAAAA020F1EAAAAEC
:10001000AAAAAA020E99AAAAAAAAAA0208B8AAAAD1
:10002000AAAAAAAAAAAAAAAAAAAAAA020B96AAAA8B
:10003000AAAAAA020FE9AAAAAAAAAAAAAAAAAAAA24
:10004000AAAAAA020800AAAAAAAAAA02069DAAAA5D
:10005000AAAAAA020800AAAAAAAAAAAAAAAAAAAAF4
:10006000AAAAAAAAAAAAAAAAAAAAAAAAAAAAAAAAF0
:10007000AAAAAAAAAAAAAAAAAAAAAAAAAAAAAAAAE0
:1000800090E6B9E0700302015B14700302020424DD
:10009000FE700302029924FB7003020155147003E1
:1000A00002014F147003020143147003020149243A
:1000B000056003020305120FEF400302031190E6EF
:1000C000BBE024FE602C14604724FD6016146031F0
:1000D00024067065E52490E6B3F0E52590E6B4F0DB
:1000E000020311E52C90E6B3F0E52D90E6B4F002A2
:1000F0000311E52690E6B3F0E52790E6B4F002039D
:1001000011E52890E6B3F0E52990E6B4F00203117A
:1001100090E6BAE0FF120EF2AA06A9077B01EA49AF
:10012000600DEE90E6B3F0EF90E6B4F002031190AC
:10013000E6A0E04401F002031190E6A0E04401F0E3
:10014000020311120FB2020311120FE10203111286
:100150000FD9020311120FA0020311120FF1400375
:1001600002031190E6B8E0247F602B14603C240267
:1001700060030201FAA200E433FF25E0FFA204E4D9
:10018000334F90E740F0E4A3F090E68AF090E68BDE
:100190007402F0020311E490E740F0A3F090E68AC5
:1001A000F090E68B7402F002031190E6BCE0547EFE
:1001B000FF7E00E0D3948040067C007D0180047CBB
:1001C000007D00EC4EFEED4F24CFF582740F3EF51E
:1001D00083E493FF3395E0FEEF24A1FFEE34E68F36
:1001E00082F583E0540190E740F0E4A3F090E68AC2
:1001F000F090E68B7402F002031190E6A0E0440157
:10020000F0020311120FF3400302031190E6B8E06D
:1002100024FE601D2402600302031190E6BAE0B4DC
:100220000105C20002031190E6A0E04401F00203C0
:100230001190E6BAE0705990E6BCE0547EFF7E0073
:10024000E0D3948040067C007D0180047C007D002A
:10025000EC4EFEED4F24CFF582740F3EF583E49310
:10026000FF3395E0FEEF24A1FFEE34E68F82F583A5
:10027000E054FEF090E6BCE05480FF131313541FCB
:10028000FFE0540F2F90E683F0E04420F0020311CA
:1002900090E6A0E04401F08078120FF5507390E6EC
:1002A000B8E024FE60202402706790E6BAE0B40152
:1002B00004D200805C90E6BAE06402605490E6A04C
:1002C000E04401F0804B90E6BCE0547EFF7E00E00D
:1002D000D3948040067C007D0180047C007D00EC8E
:1002E0004EFEED4F24CFF582740F3EF583E493FF6D
:1002F0003395E0FEEF24A1FFEE34E68F82F583E034
:100300004401F0800C120FF7500790E6A0E0440182
:10031000F090E6A0E04480F022E4F517F516F5151C
:10032000F514C205C200C204C2011209667E0B7F29
:10033000008E248F25752C0B752D1275220B7523BD
:100340001C752A0B752B43752F0B75306AEE54E024
:10035000700302045D7518007519808E1A8F1BC317
:1003600074949FFF740B9ECF2402CF3400FEE48F61
:10037000138E12F511F510F50FF50EF50DF50CAF06
:1003800013AE12AD11AC10AB0FAA0EA90DA80CC381
:10039000120E335026E519250FF582E518350EF5B6
:1003A0008374CDF0E50F2401F50FE4350EF50EE46E
:1003B000350DF50DE4350CF50C80C4E4F50FF50EA4
:1003C000F50DF50CAF13AE12AD11AC10AB0FAA0EBC
:1003D000A90DA80CC3120E335031AE0EAF0FE51BA2
:1003E0002FF582E51A3EF583E0FDE5192FF582E54C
:1003F000183EF583EDF0EF2401F50FE43EF50EE431
:10040000350DF50DE4350CF50C80B98518248519EA
:100410002574002480FF740B34FFFEC3E52D9FF587
:100420002DE52C9EF52CC3E5279FF527E5269EF5A7
:1004300026C3E5299FF529E5289EF528C3E5239FD6
:10044000F523E5229EF522C3E52B9FF52BE52A9E99
:10045000F52AC3E5309FF530E52F9EF52FD2E8430E
:10046000D82090E668E04409F0E04402F090E65EAF
:10047000E0440CF043E80443E80290E6507404F0D2
:10048000000000E4F5B290E67AF043B288F58043CC
:10049000A82E438804438910758B6F758DFE90E6F6
:1004A0008F04F075AF07759DE1E4F59E90E65CE082
:1004B000443DF0D2AF90E680E020E105D207120E75
:1004C0006A90E680E04408F00000000000000000B0
:1004D00000E054F7F0538EF8C20530010512008099
:1004E000C201300529120AFE5024C2051207DB2082
:1004F000001690E682E030E704E020E1EF90E6822B
:10050000E030E604E020E0E4120EC6120FED120F18
:10051000F980C7C0E0C0F0C083C082C0D075D000F1
:10052000C000C001C002C003C004C005C006C007AF
:10053000759AE7759B80759DE130060302061A7572
:100540000A00750B0090E67BE0FF7432250BF8A6DD
:1005500007050BE50B7002050AE59B2480C3940692
:1005600040E3E532120E4405F900058908059F10A5
:1005700005DF2005B93005D240061250060A600595
:10058000DACC05CCFF0000061A159B5391EF90E6DC
:100590005F7408F090E68DE4F0120D8A0206827412
:1005A000FD259BF59B5391EF90E65F7408F090E674
:1005B0008DE4F0120D8A02068290E7C0740AF0A35F
:1005C000E580F090E68F7402F00206745380F70223
:1005D000067490E68F7401F08040753900803B907E
:1005E000E7C074DDF0A37431F0A3742EF0A3743867
:1005F000F090E68F7404F0807B53A8F785368A75F7
:10060000CDFE75CC6F759E00801090E618740DF0CD
:10061000806290E618740CF0805A90E67BE090E6D9
:100620007CF0E59B2480FF90E68DE0FEEFC39E40CA
:10063000E9E53324FEFFE59EC39F5006E4F0D206B1
:100640008032C206759DE1759E00438902758E0059
:10065000858A8C75C800E5367006E53542808005D0
:10066000E535F4528043800890E67CE0F538438815
:100670001043C8045391EF90E65F7408F090E68D44
:10068000E4F0D007D006D005D004D003D002D001CA
:10069000D000D0D0D082D083D0F0D0E032C0E0C043
:1006A00083C082C0D075D000C000C004C005C006A1
:1006B000C0075391DF90E678E05404FF7E003002DB
:1006C0000BE0F430E1067C007D0180047C007D00BD
:1006D000EC4EFEED4F4E6008E4FF120A0F0207C811
:1006E000E53224F860030207C8E53314604904606A
:1006F000030207C8E59B2480FFBF050B059B90E61E
:1007000079E534F00207C8E5372406FFE433FEAD8F
:100710009BED2480FDE434FFFCC3ED9FEE6480F884
:10072000EC648098500B90E67BE090E679F002074D
:10073000C8120A060207C8E536701CE59B2480C370
:100740009406500B059B90E679E534F00207C875D6
:100750003601120D8A807130020F90E679E075083B
:1007600000F509C202059B805FE5372406FFE433EC
:10077000FEAD9BED2480FDE434FFFCC3ED9FEE64F1
:1007800080F8EC648098503DE5372405FFE59B2414
:1007900080B5071490E678E04440F090E679E09068
:1007A000E67BF07F01120A0FE5372404FFE59B2466
:1007B00080B5070790E678E04420F090E679E09075
:1007C000E67BF08003120A06D007D006D005D004DD
:1007D000D000D0D0D082D083D0E03290E682E04406
:1007E000C0F090E681F04387010000000000227411
:1007F00000F58690FDA57C05A3E582458370F9226E
:10080000020AE600020F8A00020F7400020F5C0069
:10081000020DC500020DFC00020FFA00020FFB00E2
:10082000020FFC00020FFD00020CAF0002051300D6
:10083000020FFE00020FFF00021000000210010074
:1008400002100200020FFB0002100300021004005D
:100850000210050002100600021007000210080036
:1008600002100900020FFB00020FFB00020FFB0049
:1008700002100A0002100B0002100C0002100D0002
:10088000020F3F0002100E0002100F0002101000B5
:1008900002101100021012000210130002101400C6
:1008A00002101500021016000210170002101800A6
:1008B0000210190002101A00C0E0C083C082C0D02C
:1008C0005388BF758B6F758DFEE59EC3947A507209
:1008D000300313E58020E10E43800890E67CE53884
:1008E000F0753800C203200313E58030E10E538019
:1008F000F790E67CE538F0753800D203E538F470FF
:100900003AE59EC3947A503390E67CE538F075382A
:1009100000E4F00521E52194004020E59E94185064
:100920001A759E00752100753800B2035388BF7593
:100930003D0090E65EE04404F080224388400538A4
:10094000801B53A8F75388F75388BF753800C2033C
:10095000752100753D0290E65EE04404F0D0D0D0F1
:1009600082D083D0E03290E60B7403F00000009058
:10097000E6047480F00000007402F000000014F03F
:10098000000000E4F000000090E6007412F090E631
:10099000017443F090E61074A0F090E68D7401F0BD
:1009A00090E61174A0F000000090E618740DF000BD
:1009B000000090E6137420F090E614F090E615F035
:1009C00090E61274E0F0000000E490E602F000000F
:1009D0000090E603F090E670F000000090E609F069
:1009E00000000090E6207402F0000000E490E62190
:1009F000F000000090E630749AF0000000E490E609
:100A000031F00000002290E678E04440F07F01EFF2
:100A100014603E046003020A9F90E7C074FFF0A3D5
:100A2000E59BF090E678E090E7C2F090E678E0F49D
:100A300030E604E04440F0E490E679F00000000085
:100A4000000090E678E090E7C3F090E68F7405F040
:100A500022E533700D90E7C07410F090E68F7401BA
:100A6000F022759B80759DE7759EC090E67BE090B7
:100A7000E67CF0E5372406FFE433FEAD9BED2480F1
:100A8000FDE434FFFCC3ED9FEE6480F8EC648098D5
:100A900040D9E537240690E68FF05380F7D2022242
:100AA0008E1C8F1D90E600E054187012E51D240185
:100AB000FFE4351CC313F51CEF13F51D801590E6FC
:100AC00000E05418FFBF100BE51D25E0F51DE51CE7
:100AD00033F51CE51D151DAE1C7002151C4E60057E
:100AE0001207EF80EE22C0E0C083C082D201539192
:100AF000EF90E65D7401F0D082D083D0E032D32253
:100B0000120100020000004047050210000001022F
:100B100000010A060002000000400100090227004F
:100B2000010100A0320904000003FF0000000705D6
:100B30000102400000070581024000000705820213
:100B400000020009022700010100A0320904000090
:100B500003FF0000000705010240000007058102B5
:100B6000400000070582020002000403090410038C
:100B70004E0065007800740063006F006D0016037E
:100B8000480044002D00550053004200200044005E
:100B9000560052000000C0E0C083C082C0D053C8DD
:100BA000FBE538D39400400D75CDFE75CC6F15383C
:100BB00043C8048062E59EC39533502790E67CE0ED
:100BC000F538E58830E40AE535F452805388EF8043
:100BD00007E535428043881075CDFE75CC6F43C85C
:100BE000048034759E00E537B47719753700759D1C
:100BF000E1059E75380075CDFE75CC6F43881043B6
:100C0000C80480135388EF53C8FB90E68DE4F0E5E9
:100C100035F4528043A80853C87FD0D0D082D08307
:100C2000D0E032787FE4F6D8FD75813D020C6A028F
:100C30000319E493A3F8E493A34003F68001F208B8
:100C4000DFF48029E493A3F85407240CC8C333C409
:100C5000540F4420C8834004F456800146F6DFE474
:100C6000800B0102040810204080900FC4E47E0134
:100C70009360BCA3FF543F30E509541FFEE493A3E7
:100C800060010ECF54C025E060A840B8E493A3FAF9
:100C9000E493A3F8E493A3C8C582C8CAC583CAF085
:100CA000A3C8C582C8CAC583CADFE9DEE780BEC063
:100CB000E0C0F0C083C082C0D075D000C000C001C9
:100CC000C002C003C004C005C006C00790E65F7440
:100CD00004F05391EF300605120D288030E53D7089
:100CE00005F59E43A808438008E53D6401601EE5C4
:100CF0003DB40205120D28801490E7C074CCF0A317
:100D0000E539F0A3E580F090E68F7440F0D007D08D
:100D100006D005D004D003D002D001D000D0D0D06E
:100D200082D083D0F0D0E032759AE720062AE49092
:100D3000E7C0F0A3E59EF0A374A0F0A37402F0A3B3
:100D40007497F0E4A3F0759BC6F59E90E7C1E0D3DD
:100D5000943A400CD2068008759BC0C206759E3A34
:100D600090E7C1E0FF90E67CE090E67BF0AE9BEE82
:100D7000C3748094815006E59EC39F40E890E68F3F
:100D80007440F05380F7E4F53D2290E678E0F430CB
:100D9000E62DE04480F0E53224F0601C2408702445
:100DA000E533B4010CE536B4010790E67974A1F09F
:100DB0002290E67974A0F02290E679E534F022E4FE
:100DC000FF120A0F22C0E0C083C08290E680E030AC
:100DD000E70E852226852327852A28852B29800C46
:100DE000852A26852B278522288523295391EF9054
:100DF000E65D7410F0D082D083D0E032C0E0C083D2
:100E0000C08290E680E030E70E8522268523278584
:100E10002A28852B29800C852A26852B27852228A0
:100E20008523295391EF90E65D7420F0D082D08322
:100E3000D0E032EB9FF5F0EA9E42F0E99D42F0E807
:100E40009C45F022D083D082F8E493701274019311
:100E5000700DA3A393F8740193F5828883E47374EF
:100E600002936860EFA3A3A380DF30070990E680B8
:100E7000E0440AF0800790E680E04408F07FDC7EE2
:100E800005120AA090E65D74FFF090E65FF05391C2
:100E9000EF90E680E054F7F022C0E0C083C082C04B
:100EA000D0E59EC3947A501543884043800890E66D
:100EB0008FE4F090E65EE054FBF0753D01D0D0D0B9
:100EC00082D083D0E03290E682E030E004E020E699
:100ED0000B90E682E030E119E030E71590E680E023
:100EE0004401F07F147E00120AA090E680E054FED8
:100EF000F022A907AE2FAF308F828E83A3E0640368
:100F00007017AD0119ED7001228F828E83E07C0095
:100F10002FFDEC3EFEAF0580DF7E007F0022C0E0AB
:100F2000C0D0E536D394004011E58055356007E523
:100F300035F452808004E5354280D0D0D0E032C014
:100F4000E0C083C0825380F77539015391BF90E6AA
:100F500051E054FEF0D082D083D0E032C0E0C083B4
:100F6000C082D2055391EF90E65D7408F0D082D034
:100F700083D0E032C0E0C083C0825391EF90E65D41
:100F80007404F0D082D083D0E032C0E0C083C0824D
:100F90005391EF90E65D7402F0D082D083D0E032BE
:100FA00090E740E53CF0E490E68AF090E68B04F0B0
:100FB000D32290E740E531F0E490E68AF090E68BAA
:100FC00004F0D322C182013D00C1060139000000B6
:100FD00001020203030404050590E6BAE0F53CD3E0
:100FE0002290E6BAE0F531D32253D8EF32D322D3A0
:100FF00022D322D322D322D32222323232323232AD
:1010000032323232323232323232323232323232C0
:101010003232323232323232323232AAAAAAAAAA58
:10102000AAAAAAAAAAAAAAAAAAAAAAAAAAAAAAAA20
:10103000AAAAAAAAAAAAAAAAAAAAAAAAAAAAAAAA10
:10104000AAAAAAAAAAAAAAAAAAAAAAAAAAAAAAAA00
:10105000AAAAAAAAAAAAAAAAAAAAAAAAAAAAAAAAF0
